:020000040800F2
:10000000A80800204901000829110008251100084E
:1000100000000000000000000000000000000000E0
:10002000000000000000000000000000AD13000808
:10003000B508000800000000A5110008AF13000873
:100040005D0100085D0100085D0100085D01000818
:100050005D0100085D0100085D0100085D01000808
:100060005D0100085D0100085D0100085D010008F8
:100070005D0100085D010008000000005D0100084E
:10008000000000005D01000800000000000000000A
:100090005D010008000000005D0100085D0100082E
:1000A0005D0100085D0100085D0100085D010008B8
:1000B0005D0100085D0100085D0100085D010008A8
:1000C00000F002F800F030F80CA030C8083824180E
:1000D0002D18A246671EAB4654465D46AC4201D180
:1000E00000F022F87E460F3E0FCCB6460126334282
:1000F00000D0FB1AA246AB4633431847AC4D000074
:10010000CC4D00000023002400250026103A01D326
:1001100078C1FBD8520700D330C100D50B607047BF
:100120001FB51FBD10B510BD00F0DCF81146FFF77C
:10013000F7FF01F015FB00F0F4F803B4FFF7F2FF4E
:1001400003BC00F0FBF8000008488047084800475F
:10015000FEE7FEE7FEE7FEE7FEE7FEE7FEE700005C
:1001600004480549054A064B70470000B9130008CA
:10017000C1000008A8020020A8080020A804002050
:10018000A8040020002203098B422CD3030A8B42CF
:1001900011D300239C464EE003460B433CD400227F
:1001A00043088B4231D303098B421CD3030A8B4291
:1001B00001D394463FE0C3098B4201D3CB01C01A5F
:1001C000524183098B4201D38B01C01A524143092A
:1001D0008B4201D34B01C01A524103098B4201D318
:1001E0000B01C01A5241C3088B4201D3CB00C01A85
:1001F000524183088B4201D38B00C01A52414308FD
:100200008B4201D34B00C01A5241411A00D2014621
:100210005241104670475DE0CA0F00D049420310BA
:1002200000D34042534000229C4603098B422DD309
:10023000030A8B4212D3FC22890112BA030A8B42B1
:100240000CD3890192118B4208D3890192118B4200
:1002500004D389013AD0921100E08909C3098B4285
:1002600001D3CB01C01A524183098B4201D38B01C8
:10027000C01A524143098B4201D34B01C01A52416B
:1002800003098B4201D30B01C01A5241C3088B42B0
:1002900001D3CB00C01A524183088B4201D38B009B
:1002A000C01A5241D9D243088B4201D34B00C01A25
:1002B0005241411A00D20146634652415B1010463A
:1002C00001D34042002B00D54942704763465B1082
:1002D00000D3404201B50020C046C04602BD704771
:1002E00070477047754600F025F8AE460500694630
:1002F0005346C008C000854618B020B5FFF730FF50
:1003000060BC00274908B6460026C0C5C0C5C0C5A8
:10031000C0C5C0C5C0C5C0C5C0C5403D49008D46AB
:10032000704710B50446C046C0462046FFF705FF9B
:1003300010BD000000487047440200200149182009
:10034000ABBEFEE726000200704770B58C1805783A
:10035000401C6B075B0F01D10378401C2A1106D1AA
:100360000278401C03E00678401C0E70491C5B1E9E
:10037000F9D12B0705D40023521E0DD40B70491C54
:10038000FAE70378401CCB1A921C03E01D780D702D
:10039000491C5B1C521EF9D5A142D8D3002070BD68
:1003A00070B5044600250A4800681123AB220021DD
:1003B00086680846B04700BF05E0E0B2044A12680C
:1003C000516888476D1C03488542F6D370BD000014
:1003D000B8010020180C000070B505460E46144602
:1003E00020462038C4B208480068C0880649096819
:1003F00089884843604304490968096842183146BE
:10040000284600F059FA70BDB4010020FFB585B050
:100410000446154601200490002700260020039082
:10042000029500E0761C02980178401C0290002999
:10043000F8D100F093F801902A480068818801986B
:10044000FFF7A0FE03900898012804D002280FD0DF
:10045000032818D10AE00398801B2249096889887B
:1004600048434008001980B204900EE004940CE068
:100470000398801B1B4909688988484361424018DA
:1004800080B2049001E0049400BF00BF0EE02A781F
:1004900006990498FFF7A0FF124800688188049825
:1004A000081880B204906D1C781C87B200F056F8D2
:1004B0000C49096889887943401A80B2094909685A
:1004C0008988884201D3012000E000202978002992
:1004D00001D0012100E0002108400028D7D109B057
:1004E000F0BD0000B4010020FFB581B00546144600
:1004F0002646E017800F8019811002980818401EC8
:1005000083B204982818401E82B213480068876896
:1005100028460299B84710480068C069002809D0E9
:100520000A9800900C480068C66922462846049B39
:100530000299B04700F01AF880B2009000F00EF86F
:1005400086B2054800688768324600210846009B4D
:10055000B84705B0F0BD0000B801002010B5024951
:1005600009684869804710BDB801002010B50249EC
:1005700009688869804710BDB801002010B50124C2
:100580000848094908600948094908600968086875
:100590008047FF20FFF704FF064800F029F80024F9
:1005A000204610BD9C010020B4010020BC010020A9
:1005B000B8010020A401002010B50B490968C868E3
:1005C000804700BFFF2101310520000700F05CFBE0
:1005D0000028F7D101220421044800F05EFB0A2024
:1005E00000F0A0F910BD0000B80100200004005088
:1005F0000149086070470000B401002010B50446AE
:100600006200044B995AA200034B985800F03CFB3F
:1006100010BD00007C1800089001002030B585B0A6
:1006200004460D461A48C06A012108431849C862A9
:10063000002D0ED160001749085A0090002001904B
:10064000022002900390A100134A5058694600F01E
:1006500025FA012D19D160000E49085A009000209A
:1006600002900E480190A1000B4A5058694600F0D4
:1006700015FA0B49095D48B20022032100F058FB2E
:100680000749095D48B200F047FB05B030BD0000E6
:10069000001002407C18000890010020000021108A
:1006A0007E18000808B5FF20FFF77AFE032315A285
:1006B0000E210A20FFF7AAFE032315A20B211C20FE
:1006C000FFF7A4FE022313A20E210A20FFF79EFECD
:1006D00002230FA20B211C20FFF798FE104836239F
:1006E0001422032100900A20FFF7FEFE0C48362357
:1006F0001422032100906C20FFF7F6FEFFF75CFF49
:1007000008BD0000427574746F6E20310000000057
:100710004F666600427574746F6E203200000000F0
:100720000000002008B5FF20FFF73AFE032315A2C2
:100730000E210A20FFF76AFE032315A20B211C20BD
:10074000FFF764FE022313A20E210A20FFF75EFECC
:10075000022313A20B211C20FFF758FE1148362359
:100760001422032100900A20FFF7BEFE0E48362314
:100770001422032100906C20FFF7B6FEFFF71CFF48
:1007800008BD0000427574746F6E203100000000D7
:100790004F666600427574746F6E20320000000070
:1007A0004F6E000000000020A200002008B5FF20CE
:1007B000FFF7F6FD032315A20E210A20FFF726FE00
:1007C000032315A20B211C20FFF720FE022313A2F6
:1007D0000E210A20FFF71AFE022313A20B211C2070
:1007E000FFF714FE114836231422032100900A203B
:1007F000FFF77AFE0E4836231422032100906C2066
:10080000FFF772FEFFF7D8FE08BD00004275747452
:100810006F6E2031000000004F6E0000427574744E
:100820006F6E2032000000004F666600A2000020BC
:100830000000002008B5FF20FFF7B2FD032315A23A
:100840000E210A20FFF7E2FD032315A20B211C2035
:10085000FFF7DCFD022313A20E210A20FFF7D6FDCD
:1008600002230FA20B211C20FFF7D0FD10483623D6
:100870001422032100900A20FFF736FE0C4836238D
:100880001422032100906C20FFF72EFEFFF794FE48
:1008900008BD0000427574746F6E203100000000C6
:1008A0004F6E0000427574746F6E203200000000BD
:1008B000A200002070470000F7B584B005460E4640
:1008C0000024002003900290019014480068808862
:1008D000019012480068C088029002983018401EAB
:1008E00083B201982818401E82B20D480068314634
:1008F00087682846B847019902984843039000BF8B
:1009000006E0069A105D064A126851688847641C22
:1009100003988442F5D307B0F0BD0000B401002075
:10092000B801002010B50446204600F0A9F810BD1B
:1009300000B585B03548C06A012108433349C86213
:100940000846C06A022108433049C8620846C06AA6
:10095000022108432D49C8620846C06A01210843A4
:100960002A49C8620846C06A022108432749C8626A
:100970000120C0030090012001900020029003207C
:10098000039069460520000700F088F80120C002A6
:10099000009069461E4800F081F8042000906946E6
:1009A0001B4800F07BF8012080020090694618483F
:1009B00000F074F8FF200130009000200190022028
:1009C000029069460520000700F068F80022012126
:1009D00089020F4800F061F900220121C9030520B6
:1009E000000700F05AF90122D1030520000700F0AA
:1009F00054F901220421064800F04FF90A20FFF7BC
:100A000091FF00F067FC05B000BD0000001002403F
:100A10000004005010B5044600220121C90305203E
:100A2000000700F03AF90122D102064800F035F93A
:100A3000E0B200F0A9FC0122D1030520000700F07C
:100A40002CF910BD0004005010B50446002201210D
:100A5000C9030520000700F020F900220121C90286
:100A6000064800F01AF9204600F08EFC0122D1035E
:100A70000520000700F011F910BD0000000400502F
:100A800031B5002400F010F9044600BF00F00CF965
:100A9000001B00998842F9D338BD0000F0B5034629
:100AA0000A460027002400200021DAE001258D40BD
:100AB0002F4615683D402C46BC4276D15568022D24
:100AC00002D05568122D15D1CD08AD001E46203636
:100AD00070594D07EE0E0F25B5400646AE43304621
:100AE0004E07F60E1569B5402843CD08AE001D46E9
:100AF0002035A8515568012D08D05568022D05D024
:100B00005568112D02D05568122D18D198684E00E5
:100B10000325B5400646AE4330464E00D568B54085
:100B200028439860586801258D400646AE433046FC
:100B30001026556835402D098D40284358601868A7
:100B40004E000325B5400646AE4330461579AD0745
:100B5000AD0F4E00B54028431860D8684E000325FD
:100B6000B5400646AE4330464E009568B540284332
:100B7000D8600126360755683540B54270D13B4DE7
:100B80006D6B01263543394E7563394D8E08B600BD
:100B9000A8598D072E0F0F25ED43B5402840052598
:100BA0002D07AB4202D1002515E059E0314DAB4293
:100BB00001D101250FE0304DAB4201D102250AE001
:100BC0002E4DAB4201D1032505E02D4DAB4201D1A5
:100BD000042500E005258E07360FB5402843244D37
:100BE0008E08B600A851274D28680546A54328461B
:100BF0000126360455683540B54202D105462543E5
:100C00002846204D286068680546A54328460126E9
:100C1000760455683540B54202D10546254328463D
:100C2000184D6860A8680546A54328460126360584
:100C300055683540B54202D1054625432846114D39
:100C4000A860E8680546A54328460126760555684C
:100C50003540B54202D1054625432846094DE86096
:100C6000491C102900D221E7F0BD0000001002400D
:100C7000080001400004005000080050000C005023
:100C8000001C005000040140024613690B40002B79
:100C900001D0012000E000207047002A01D08161CE
:100CA00000E0816270470000014800687047000062
:100CB0004801002002480068401C01490860704754
:100CC0004801002010B50948006840210843074941
:100CD00008600846006802210843044908600320B0
:100CE00000F006F800F017F8002010BD00200240C8
:100CF00070B5044600F026F806467D21C900FFF7CE
:100D000041FA054600F0F2F900222146501E00F09B
:100D10000FF8002070BD704700BFC206D20E01213F
:100D20009140024A116000BF7047000000E100E0FE
:100D300070B504460D4616462946204600F0F6F9E1
:100D400070BD000010B500F013F80649C968F02224
:100D500011400909044A515CC8400449086008462A
:100D6000006810BD001002405501002068010020FD
:100D7000F8B500240027002000900025002629480F
:100D80004068072149030840450BA80026490D5833
:100D90002448C0680C210840002806D0042806D04A
:100DA00008280ED00C2838D10DE02E4637E01D481B
:100DB000006810210840002801D01C4E00E01C4EA5
:100DC0002DE01C4E2BE01748C0680F218904084015
:100DD00004461448C0680321890508400746A00C52
:100DE00015490C5CB80D471C0E48C0680121090468
:100DF000084000900098002807D10D49614308463B
:100E00003946FFF7BFF9064606E00A49614308463E
:100E10003946FFF7B7F9064601E02E4600BF00BF8E
:100E20003046F8BD001002405C18000800093D0083
:100E30000024F40000127A004C01002010B5044692
:100E4000002C01D1012010BD022151200155206844
:100E500000684021884321680860204600F054F86B
:100E60000021522001555120015500BF502001554D
:100E700000BF0020E7E701465120405C704710B5F5
:100E80000446002C01D1012010BD5120005D002836
:100E900002D1204600F039F8022151200155206886
:100EA00000684021884321680860A16860680843A1
:100EB000E16808432169084361690843012252023D
:100EC000A16911400843E1690843216A0843A16A06
:100ED000084321680860A069000C04210840616A89
:100EE0000843216848602168E06A08612068C06999
:100EF000910088432168C8610021522001550121D9
:100F0000512001550020BFE770477047F8B50446EF
:100F10000E4615461F465120005D01287CD1002E4B
:100F200001D0002D01D10120F8BD00BF5020005D8F
:100F3000012801D10220F7E701215020015500BF0F
:100F40001221512001550021522001552663A5860A
:100F5000E5860020E064A064A087E08701214903C2
:100F6000A06A88420DD100BF2068006888432168CC
:100F7000086020680068012149030843216808606F
:100F800000BF0121C903A068884205D1206800681C
:100F90004910084321680860206800684021084023
:100FA000402804D020680068084321680860E06891
:100FB000002832D16068002802D0E08E012808D1D4
:100FC000216B481C206308782168C860E08E401EB1
:100FD000E08612E03B4600220221204600F0E3F8C2
:100FE000002801D003209FE7216B481C206308786C
:100FF0002168C860E08E401EE086E08E0028E9DCB3
:1010000001214903A06A88423AD12068006849104A
:1010100008432168086033E065E06068002802D07A
:10102000E08E012809D1206B00882168C860206B00
:10103000801C2063E08E401EE08613E03B460022C9
:101040000221204600F0AFF8002801D003206BE712
:10105000206B00882168C860206B801C2063E08EB4
:10106000401EE086E08E0028E8DC01214903A06AEA
:10107000884205D12068006849100843216808604B
:101080003B4600220221204600F08DF8002807D0C0
:101090005220005D2021084352210855032043E7D8
:1010A0003B4601228021204600F07DF8002807D031
:1010B0005220005D2021084352210855032033E7C8
:1010C000A068002805D100BF2068C068206880683B
:1010D00000BF01215120015500BF002150200155C2
:1010E00000BF002020E702201EE7000070B5044684
:1010F0002546681E0949884201D901200CE0681E76
:10110000074948610321081F00F010F80020044936
:10111000886107200861002070BD0000FFFFFF000C
:1011200000E000E000BFFEE77047000010B50028B7
:1011300019DA1A4A03071B0F083B9B089B00D25879
:101140008307DC0EFF23A3409A438B071B0E840703
:10115000E40EA3401A43114B0407240F083CA408D3
:10116000A4001A5118E00E4A03231B02D218830868
:101170009B00D2588307DC0EFF23A3409A438B07C2
:101180001B0E8407E40EA3401A43054B03242402DC
:101190001B198408A4001A5110BD00001CED00E0CA
:1011A00000E100E07047FFB581B004460E461D46E1
:1011B0000027FFF779FD0746039800283FD133E069
:1011C000681C002830D0002D04D0FFF76DFDC01B37
:1011D000A84229D920684068E021884321684860F6
:1011E0002068006840218843216808600121490384
:1011F000A06A88420DD100BF20680068884321683A
:1012000008602068006801214903084321680860DC
:1012100000BF01215120015500BF00215020015580
:1012200000BF032005B0F0BD206880683040B042A8
:1012300001D1012000E000200028C1D03DE032E0D3
:10124000681C00282FD0002D04D0FFF72DFDC01BF7
:10125000A84228D920684068E02188432168486076
:101260002068006840218843216808600121490303
:10127000A06A88420DD100BF2068006888432168B9
:10128000086020680068012149030843216808605C
:1012900000BF01215120015500BF00215020015500
:1012A00000BF0320BEE7206880683040B04201D113
:1012B000012000E000200028C2D10020B2E7000099
:1012C00010B50348FFF7BAFD00F004F810BD0000A8
:1012D000F001002010B51348FFF7CDFD002820D104
:1012E000114810490860FF200530486000210D4872
:1012F00081601021C1610021C16001214161022191
:1013000001610021016201214902816100218162A4
:101310000721C1620021416200F008F80148FFF78F
:10132000AEFD10BDF00100200030014010B586B0C8
:1013300004461348C06A022108431149C8620820C4
:1013400001900220029001200390032004900020CD
:10135000059001A90B48FFF7A1FB20200190002078
:1013600005900220039001A90648FFF797FB044867
:10137000406B0121090308430149486306B010BDD1
:10138000001002400004005031B5002401231B036B
:10139000012269460448FFF7B9FD0446002C01D03C
:1013A000FFF78EFF38BD0000F0010020704710B538
:1013B000FFF780FC10BD000015480068FF210131D7
:1013C0000843134908600846C0681249084010499C
:1013D000C86008460068104908400D490860084682
:1013E0008068400840008860084600680121890440
:1013F0008843074908600846C068FD2109048843FE
:101400000349C86000200861C80304498860704728
:10141000001002400C40FF88F6FFF6FE00ED00E0F1
:1014200010B52220FFF710FB0320FFF7F3FA20206E
:10143000FFF70AFB10BDFFB585B015460024002656
:10144000002002902420FFF7FFFA2846E917490FF1
:101450000918C910C900691A4DD100273EE00E983D
:10146000C65D002E33D0002003902CE0002412E053
:10147000F007C00F002806D004A8005DFC2108403A
:1014800004A9085505E004A8005D0321084304A948
:1014900008557610641C042CEAD36946087C800148
:1014A000497C090108436946897C890008436946EB
:1014B000C97C0843C0B202900298FFF7ABFA0398C8
:1014C000401CC0B2039003980228CFDB05E0FF2048
:1014D000FFF7A0FAFF20FFF79DFA7F1CEA17920F93
:1014E00052199210089B5A431046D20F12185210EC
:1014F000BA42B4D8A0E0002790E00E98C65DE81785
:10150000800F40198010401CC20F009501901018E8
:101510004110781CFEF736FE00293ED0002E33D055
:10152000002003902CE0002412E0F007C00F0028F8
:1015300006D004A8005DFC21084004A9085505E078
:1015400004A8005D0321084304A908557610641C13
:10155000042CEAD36946087C8001497C09010843D0
:101560006946897C890008436946C97C0843C0B242
:1015700002900298FFF74EFA0398401CC0B2039005
:1015800003980228CFDB48E0002E46D1FF20FFF76A
:1015900041FAFF20FFF73EFA3FE0E817800F4019BD
:1015A0008010401CC20F0095019010184110781C4B
:1015B000FEF7E8FD002930D1F02E29D0002412E0FA
:1015C000F007C00F002806D004A8005DFC210840E9
:1015D00004A9085505E004A8005D0321084304A9F7
:1015E00008557610641C042CEAD36946087C8001F7
:1015F000497C090108436946897C8900084369469A
:10160000C97C0843C0B202900298FFF703FA04E0D5
:10161000F02E02D1FF20FFF7FDF97F1CEA17920F91
:1016200052199210521C089B5A431046D20F12189E
:101630005210BA4200D960E709B0F0BD12207047DD
:10164000AC20704710B50024FFF772F91020FFF7A7
:10165000FBF90020FFF7DEF91120FFF7F5F9032071
:10166000FFF7D8F94420FFF7EFF90020FFF7D2F990
:101670001120FFF7CFF94520FFF7E6F90020FFF72B
:10168000C9F9AB20FFF7C6F94E20FFF7DDF90020BE
:10169000FFF7C0F94F20FFF7D7F90020FFF7BAF99D
:1016A000F020FFF7D1F91F20FFF7B4F92120FFF751
:1016B000CBF90320FFF7AEF92C20FFF7C5F9A020E6
:1016C000FFF7A8F93C20FFF7BFF96420FFF7A2F964
:1016D0003220FFF7B9F900BF05E00449085DFFF7C4
:1016E00099F9601CC4B25A2CF7DB10BD4E4E0008AD
:1016F00010B52220FFF7A8F9C420FFF78BF92020AE
:10170000FFF7A2F910BDF8B507460C4615461E4670
:101710004420FFF799F92046FFF77CF93046FFF7A0
:1017200079F94520FFF790F93846FFF773F9284615
:10173000FFF770F94E20FFF787F92046FFF76AF9A7
:101740004F20FFF781F93846FFF764F9F8BD10B56F
:1017500004462420FFF778F92046FFF75BF910BD17
:10176000FFF7B0FAFEF70AFF00210846FEF756FF22
:101770003748C06A012108433549C862022035490B
:1017800008600020486002208860C86005200007CB
:10179000FFF784F90022042105200007FFF77DFAF6
:1017A000FEF780FF53E00020FEF728FF00280FD14E
:1017B0002948006800280BD0022105200007FFF708
:1017C00063FA002804D1FEF76DFF0020224908606B
:1017D0000020FEF713FF01280FD11F4800680128E1
:1017E0000BD0022105200007FFF74EFA002804D194
:1017F000FEF7DCFF0120184908600020FEF7FEFE1E
:1018000000280FD11448006802280BD002210520BF
:101810000007FFF739FA012804D1FEF783FF022001
:101820000D4908600020FEF7E9FE01280FD10A48A3
:10183000006803280BD0022105200007FFF724FAD7
:10184000012804D1FEF7F6FF032003490860AAE748
:1018500000100240DC0100204401002000FA0000DA
:1018600000F4010000E8030000D0070040420F0030
:1018700080841E0000093D0010002000010005FFCB
:10188000FFFFFFFFFFFFFFFFFFFFFFFFFFFFFFFF68
:10189000FFFFFFFFFFFFFFFFFFFFFFFFFFFFFFFF58
:1018A000FFFFFFFFFFFFFFFFFFFFFFFFFFFFFFFF48
:1018B000FFFFFFFFFFFFFFFFFFFFFFFFFFFFFFFF38
:1018C000FFFFFFFFFFFFFFFFFFFFFFFFFFFFFFFF28
:1018D000FFFFFFFFFFFFFFFFFFFFFFFFFFFFFFF027
:1018E000FF0003FFF0F00003FFF0FF0003FFFFFF26
:1018F000FFFFFFFFFFFFFFFFFFFFFFFFFFFFFFFFF8
:10190000FFFFFFFFFFFFFFFFFFFFFFFFFFFFFFFFE7
:10191000FFFFFFFFFFFFFFFFFFFFFFFFFFFC0FFFCA
:10192000FFFF000FFFFFFFFC0FFFFFFFFFFFFFFFA9
:10193000FFFFFFFFFFFFFC0FFFFFFF000FFFFFFF99
:10194000FC0FFFFFFFFFFFFFFFFFFFFFFFFFFFFF9A
:10195000FFFFFFFFFFFFFFFFFFFFFFFFFFC3C3FF0F
:10196000FFFFC3C3FFFF00000000FF00000000FFF7
:10197000FFC3C3FFFFFFC3C3FFFF00000000FF0062
:10198000000000FFFFC3C3FFFFFFC3C3FFFFFFFF54
:10199000FFFFFFFFFFFFFFFFFFFFFFFFFFFFFFFF57
:1019A000FFFFFFFFFFFFFFFC03C0FFFFFC03003F43
:1019B000FFFC3F0F0FFF003F0F00FF003F0F00FF36
:1019C000FC3C3F0FFFFF003C0FFFFFC0FC0FFFFF81
:1019D000FFFFFFFFFFFFFFFFFFFFFFFFFFFFFFFF17
:1019E000FFFFFFFFFFFFFFFFFFF0FC0FFFFFF0F324
:1019F000F3FFFFFC33F3FFFFFC33F3FFFC0F3C0F5F
:101A0000FFF3F30FFFFFF3F30FFFFFF3F3C3FFFF4A
:101A1000FC0FC3FFFFFFFFFFFFFFFFFFFFFFFFFF05
:101A2000FFFFFFFFFFFFFFFFFFFFFFFFFFFFFFFFC6
:101A3000FFFFFFFC03FFFFFFFC00C0FFFFF0F00013
:101A4000FFFFF0F03C3FFFF0C0FC3FFFF003FC3F26
:101A5000FFFC03FC3FFFF0C0FC3FFFF0F0FC3FFF4A
:101A6000FFFFFFFFFFFFFFFFFFFFFFFFFFFFFFFF86
:101A7000FFFFFFFFFFFFFFFFFFFFFFFFFFFFFFFF76
:101A8000FFFFFFFFFFFFFFFFFFFFFC0FFFFFFF0058
:101A90000FFFFFFFFC0FFFFFFFFFFFFFFFFFFFFF39
:101AA000FFFFFFFFFFFFFFFFFFFFFFFFFFFFFFFF46
:101AB000FFFFFFFFFFFFFFFFFFFFFFFFFFFFFFFF36
:101AC000FFFFFFFFFFFFFFFFFFFFFFFFFFFFFF0025
:101AD0000FFFFFC000003FFC00FFF003FC3FFFFFD3
:101AE000C3FFFFFFFFFFFFFFFFFFFFFFFFFFFFFF42
:101AF000FFFFFFFFFFFFFFFFFFFFFFFFFFFFFFFFF6
:101B0000FFFFFFFFFFFFFFFFFFFC3FFFFFC3FC00E6
:101B1000FFF003FFC000003FFFFF000FFFFFFFFFCC
:101B2000FFFFFFFFFFFFFFFFFFFFFFFFFFFFFFFFC5
:101B3000FFFFFFFFFFFFFFFFFFFFFFFFFFFFFFFFB5
:101B4000FFFFFFFFFFFFFFFFFFFFFFFFFFF0FFFFB4
:101B5000FFF0F0FFFFFFF003FFFFFFFC0003FFFFBC
:101B6000FC0003FFFFF003FFFFFFF0F0FFFFFFFFAC
:101B7000F0FFFFFFFFFFFFFFFFFFFFFFFFFFFFFF84
:101B8000FFFFFFFFFFFFFFFFFFFFFFFFFFFC3FFF28
:101B9000FFFFFC3FFFFFFFFC3FFFFFFFFC3FFFFF9E
:101BA000FC00003FFFFC00003FFFFFFC3FFFFFFF8A
:101BB000FC3FFFFFFFFC3FFFFFFFFC3FFFFFFFFF7E
:101BC000FFFFFFFFFFFFFFFFFFFFFFFFFFFFFFFF25
:101BD000FFFFFFFFFFFFFFFFFFFFFFFC0FFFFFFF08
:101BE000FF003FFFFFFFF03FFFFFFFFF3FFFFFFF53
:101BF000FFFFFFFFFFFFFFFFFFFFFFFFFFFFFFFFF5
:101C0000FFFFFFFFFFFFFFFFFFFFFFFFFFFFFFFFE4
:101C1000FFFFFFFFFFFFFFFFFFFC3FFFFFFFFC3F5A
:101C2000FFFFFFFC3FFFFFFFFC3FFFFFFFFC3FFF0D
:101C3000FFFFFC3FFFFFFFFC3FFFFFFFFC3FFFFFFD
:101C4000FFFC3FFFFFFFFFFFFFFFFFFFFFFFFFFF67
:101C5000FFFFFFFFFFFFFFFFFFFFFFFFFFFFFFFF94
:101C6000FFFFFFFFFFFFFFFFFFFFFFFFFFFFFFFF84
:101C7000FFFFF03FFFFFFFF03FFFFFFFF03FFFFFE1
:101C8000FFFFFFFFFFFFFFFFFFFFFFFFFFFFFFFF64
:101C9000FFFFFFFFFFFFFFFFFFFFFFFFFFFFFFFF54
:101CA000FFFFFFFFFFFFFFFFFF0FFFFFFFFF003FF3
:101CB000FFFFFFF003FFFFFFFFC03FFFFFFFFC033D
:101CC000FFFFFFFFC00FFFFFFFFC00FFFFFFFFF064
:101CD000FFFFFFFFFFFFFFFFFFFFFFFFFFFFFFFF14
:101CE000FFFFFFFFFFFFFFFFFFFFFFC000FFFFFC45
:101CF00000000FFFF03FFF03FFF0FFFFC3FFF0FF07
:101D0000FFC3FFF0FFFFC3FFF03FFF03FFFC000036
:101D10000FFFFFC000FFFFFFFFFFFFFFFFFFFFFF01
:101D2000FFFFFFFFFFFFFFFFFFFFFFFFFFFFFFFFC3
:101D3000FFFFFFFFFFF0FFFF0FFFF0FFFF0FFFF0C0
:101D4000FFFF0FFFF0000003FFF0000003FFF0FFB4
:101D5000FFFFFFF0FFFFFFFFF0FFFFFFFFFFFFFFB1
:101D6000FFFFFFFFFFFFFFFFFFFFFFFFFFFFFFFF83
:101D7000FFFFFFFFFFFFF0FFFC3FFFF03FFC0FFF07
:101D8000F00FFF03FFF0C3FFC3FFF0F0FFC3FFF04E
:101D9000FC3FC3FFF0FF0F03FFF0FFC00FFFF0FF9A
:101DA000F03FFFFFFFFFFFFFFFFFFFFFFFFFFFFF12
:101DB000FFFFFFFFFFFFFFFC3FFFFFFFF03FFF0FB5
:101DC000FFF0FFFF0FFFF0FFFFC3FFF0FF0FC3FFA8
:101DD000F0FF0FC3FFF0FF0FC3FFF03C0303FFFC56
:101DE00000000FFFFF00F03FFFFFFFFFFFFFFFFFBF
:101DF000FFFFFFFFFFFFFFFFFFFFFFFFFFFFFFFFF3
:101E0000FFFFFFC0FFFFFFFFC03FFFFFFFC303FF58
:101E1000FFFFC3C0FFFFF0C3FC0FFFF0C3FF03FFD2
:101E2000F0000003FFF0000003FFF0C3FFFFFFFF1F
:101E3000FFFFFFFFFFFFFFFFFFFFFFFFFFFFFFFFB2
:101E4000FFFFFFFFFFFFFFFFFC3FFFFFFFF03F0033
:101E500003FFF0FF0003FFF0FFC3C3FFF0FFC3C3A6
:101E6000FFF0FFC3C3FFF03F03C3FFFC000FC3FF3E
:101E7000FF003FFFFFFFFFFFFFFFFFFFFFFFFFFF31
:101E8000FFFFFFFFFFFFFFFFFFFFFFFFFFFFFFC0A1
:101E900003FFFFFC00003FFFFC3C300FFFF0FF0F93
:101EA0000FFFF0FF0F03FFF0FF0FC3FFF03C0FC366
:101EB000FFFC003FC3FFFF00FFC3FFFFFFFFFFFF6B
:101EC000FFFFFFFFFFFFFFFFFFFFFFFFFFFFFFFF22
:101ED000FFFFFFFFFFFFFF03FFFFFFFF03FFFFFF0A
:101EE000FFC3FFFFFFFFC3FFF03FFFC3FFF000FF93
:101EF000C3FFFFC003C3FFFFFC0003FFFFFFFC03A2
:101F0000FFFFFFFFFFFFFFFFFFFFFFFFFFFFFFFFE1
:101F1000FFFFFFFFFFFFFFFFFFFFFF00F03FFFFCA2
:101F200000000FFFF03C0303FFF0FF0FC3FFF0FFC3
:101F30000FC3FFF0FF0FC3FFF03C0303FFFC0000E3
:101F40000FFFFF00F03FFFFFFFFFFFFFFFFFFFFF5F
:101F5000FFFFFFFFFFFFFFFFFFFFFFFFFFFFFFFF91
:101F6000F0FFC03FFFF0FF000FFFF0FC0F03FFF09A
:101F7000FC3FC3FFF03C3FC3FFFC3C3FC3FFFC03FF
:101F80000F0FFFFF00000FFFFFF000FFFFFFFFFF3D
:101F9000FFFFFFFFFFFFFFFFFFFFFFFFFFFFFFFF51
:101FA000FFFFFFFFFFFFFFFFFFFFFFFFFFFFFFFF41
:101FB000FFFFFFFFFFFFFFFFFFFFF03F03FFFFF00B
:101FC0003F03FFFFF03F03FFFFFFFFFFFFFFFFFFA8
:101FD000FFFFFFFFFFFFFFFFFFFFFFFFFFFFFFFF11
:101FE000FFFFFFFFFFFFFFFFFFFFFFFFFFFFFFFF01
:101FF000FFFFFFFFFFFFFFFFFFFFF03FFFFFFFFCC3
:1020000003FFFFFFFFC3F03FFFFFF3F03FFFFFFFC2
:10201000F03FFFFFFFFFFFFFFFFFFFFFFFFFFFFF9F
:10202000FFFFFFFFFFFFFFFFFFFFFFFFFFFFFCFFC3
:10203000FFFFFFFCFFFFFFFFF03FFFFFFFF03FFF51
:10204000FFFFC30FFFFFFF0FC3FFFFFF0FC3FFFF24
:10205000FC3FF0FFFFFC3FF0FFFFF0FFFC3FFFF015
:10206000FFFC3FFFFFFFFFFFFFFFFFFFFFFFFFFF43
:10207000FFFFFFFFC3C3FFFFFFC3C3FFFFFFC3C3D8
:10208000FFFFFFC3C3FFFFFFC3C3FFFFFFC3C3FFC8
:10209000FFFFC3C3FFFFFFC3C3FFFFFFC3C3FFFFB8
:1020A000FFC3C3FFFFFFC3C3FFFFFFFFFFFFFFFF30
:1020B000FFFFFFFFFFFFFFFFFFFFFFFFFFFFF0FF3F
:1020C000FC3FFFF0FFFC3FFFFC3FF0FFFFFC3FF059
:1020D000FFFFFF0FC3FFFFFF0FC3FFFFFFC30FFF94
:1020E000FFFFF03FFFFFFFF03FFFFFFFFCFFFFFFA1
:1020F000FFFCFFFFFFFFFFFFFFFFFFFFFFFFFFFFF3
:10210000FFFFFFFFFFFFFFFFFFFFFFF03FFFFFFFAE
:10211000F00FFFF0FFFF0FFFF0F0FF0FFFF0F03FB9
:102120000FFFFFFC3F0FFFFFFF003FFFFFFFC0FF60
:10213000FFFFFFFFFFFFFFFFFFFFFFFFFFFFFFFFAF
:10214000FFFFFFFFFFFFFFFFFFFFFFFFFFFFFFFF9F
:102150000000FFFFF0FFFF0FFFCFFFFFCFFFCFF02B
:102160003FF3FFCFCFCFF3FFCFCFCFC3FFF3C000FD
:102170003FFFFFFFFFFFFFFFFFFFFFFFFFFFFFFF2F
:10218000FFFFFFFFFFFFFFFFFFFFFFF0FFFFFFFF6E
:10219000F03FFFFFFFF003FF0FFFF0C03F0FFFFF17
:1021A000C0030FFFFFC3C00FFFFFC3FC0FFFFFC340
:1021B000000FFFF0C003FFFFF000FFFFFFF03FFF45
:1021C000FFFFF0FFFFFFFFFFFFFFFFFFFFFFFFFF2E
:1021D000FFFFFFFFFFFFF0FFFF0FFFF000000FFF0B
:1021E000F000000FFFF0FC3F0FFFF0FC3F0FFFF08F
:1021F000FC3F0FFFF0FC0F0FFFF0F0003FFFF0007F
:10220000C0FFFFFC03FFFFFFFFFFFFFFFFFFFFFF1C
:10221000FFFFFFFFFFFFFFFFFFFFFFFFFFC003FF09
:10222000FFFF0000FFFFFC0FF03FFFF03FFC0FFF40
:10223000F0FFFF0FFFF0FFFF0FFFF0FFFF0FFFF0BA
:102240003FFC3FFFFC0FF00FFFFF0FF00FFFFFFF02
:10225000FFFFFFFFFFFFFFFFFFFFFFFFFFF0FFFF9D
:102260000FFFF000000FFFF000000FFFF0FFFF0F67
:10227000FFF0FFFF0FFFF0FFFF0FFFF0FFFF0FFF6B
:10228000F03FFC0FFFFC0FF03FFFFF0000FFFFFFE0
:10229000C003FFFFFFFFFFFFFFFFFFFFFFFFFFFF89
:1022A000FFFFFFFFFFFFFFFFF0FFFF0FFFF000004A
:1022B0000FFFF000000FFFF0FC3F0FFFF0FC3F0F9F
:1022C000FFF0F00F0FFFF0F00F0FFFF0FFFF0FFF19
:1022D000F00FF00FFFF00FF00FFFFFFFFFFFFFFF0A
:1022E000FFFFFFFFFFFFFFFFFFFFFFFFFFFFF0FF0D
:1022F000FF0FFFF000000FFFF000000FFFF0FC3FAA
:102300000FFFF0FC3F0FFFF0F00F0FFFF0F00F0F8B
:10231000FFFFFFFF0FFFFFFFF00FFFFFFFF00FFFBB
:10232000FFFFFFFFFFFFFFFFFFFFFFFFFFFFFFFFBD
:10233000FFFFFFFFFFC003FFFFFC00003FFFFC00AB
:10234000003FFFF0FFFF0FFFF0FFFF0FFFF0F0FF78
:102350000FFFF0F0FF0FFFF0F0FC3FFFFC00F00F6D
:10236000FFFC00F00FFFFFF0FFFFFFFFFFFFFFFF8D
:10237000FFFFFFFFFFFFFFFFFFFFF0FFFF0FFFF07B
:1023800000000FFFF000000FFFF0FC3F0FFFFFFC0D
:102390003FFFFFFFFC3FFFFFF0FC3F0FFFF000009F
:1023A0000FFFF000000FFFF0FFFF0FFFFFFFFFFF29
:1023B000FFFFFFFFFFFFFFFFFFFFFFFFFFFFFFFF2D
:1023C000FFFFFFFFFFF0FFFF0FFFF0FFFF0FFFF02A
:1023D000FFFF0FFFF000000FFFF000000FFFF0FF06
:1023E000FF0FFFF0FFFF0FFFF0FFFF0FFFFFFFFFEB
:1023F000FFFFFFFFFFFFFFFFFFFFFFFFFFFFFFFFED
:10240000FFFFFFFFFFFFFC00FFFFFFFC00FFFFFFE0
:10241000F0FFFFFFFFF0FFFFFFFFF0FFFF0FFFF0F8
:10242000FFFF0FFFF03FFF0FFFFC00000FFFFF005B
:10243000000FFFFFFFFF0FFFFFFFFF0FFFFFFFFF7B
:10244000FFFFFFFFFFFFFFFFFFFFFFFFF0FFFF0F9B
:10245000FFF000000FFFF000000FFFF0FC3F0FFF48
:10246000F0FF0F0FFFFFFC03FFFFFFC0F00FFFFCAB
:1024700003FC0FFFF03FFC0FFFF0FFFF0FFFF0FF2B
:10248000FF0FFFFFFFFFFFFFFFFFFFFFFFFFFFFF4C
:10249000FFFFF0FFFF0FFFF0FFFF0FFFF000000F47
:1024A000FFF000000FFFF0FFFF0FFFF0FFFF0FFF37
:1024B000F0FFFFFFFFF0FFFFFFFFF003FFFFFFF064
:1024C00003FFFFFFFFFFFFFFFFFFFFFFFFFFFFFF18
:1024D000FFFFFFF0FFFF0FFFF000000FFFF0000015
:1024E0000FFFF0FFF00FFFF0FC03FFFFFFC03FFF07
:1024F000FFFFC03FFFFFF0FC03FFFFF0FFF00FFF07
:10250000F000000FFFF000000FFFF0FFFF0FFFFFD4
:10251000FFFFFFFFFFFFFFFFFFFFFFFFFFFFF0FFDA
:10252000FF0FFFF000000FFFF000000FFFF0FFC0F3
:102530003FFFF0FC03FFFFFFC03F0FFFFC03FF0F57
:10254000FFF000000FFFF000000FFFFFFFFF0FFF85
:10255000FFFFFFFFFFFFFFFFFFFFFFFFFFFFFFFF8B
:10256000FFFFFFFFFFC003FFFFFF0000FFFFFC0FA7
:10257000F03FFFF03FFC0FFFF0FFFF0FFFF0FFFF0A
:102580000FFFF03FFC0FFFFC0FF03FFFFF0000FFCD
:10259000FFFFC003FFFFFFFFFFFFFFFFFFFFFFFF86
:1025A000FFFFFFFFFFFFFFFFFFFFF0FFFF0FFFF049
:1025B00000000FFFF000000FFFF0F0FF0FFFF0F042
:1025C000FF0FFFF0F0FF0FFFFFF0FF0FFFFFF03CEA
:1025D0000FFFFFFC003FFFFFFF00FFFFFFFFFFFFBC
:1025E000FFFFFFFFFFFFFFFFFFFFFFFFFFFFFFFFFB
:1025F000FFC003FFFFFF0000FFFC3C0FF03FFC00AB
:102600003FFC0FFF00FFFF0FFF00FFFF0FFC003F2D
:10261000FC0FFC3C0FF03FFC0F0000FFFF0FC0035E
:10262000FFFFFFFFFFFFFFFFFFFFFFFFFFFFFFFFBA
:10263000FFFFFFFFFFFFF0FFFF0FFFF000000FFFA6
:10264000F000000FFFF0FC3F0FFFF0FC3F0FFFFF1B
:10265000FC3F0FFFFFF03F0FFFFF000C0FFFFC03DD
:10266000003FFFF0FFC0FFFFF0FFFFFFFFFFFFFF96
:10267000FFFFFFFFFFFFFFFFFFFFFFFFF00FC0FFA8
:10268000FFF00F003FFFFC3F0C0FFFF0FC3F0FFF80
:10269000F0FC3F0FFFF0FC3F0FFFF0FC3F0FFFF09F
:1026A00030FC3FFFFC00F00FFFFF03F00FFFFFFFC8
:1026B000FFFFFFFFFFFFFFFFFFFFFFFFFFFFFFFF2A
:1026C000FFFFFFFFC00FFFFFFFC00FFFF0FFFF0F77
:1026D000FFF0FFFF0FFFF000000FFFF000000FFF03
:1026E000F0FFFF0FFFF0FFFF0FFFFFFFC00FFFFF27
:1026F000FFC00FFFFFFFFFFFFFFFFFFFFFFFFFFF19
:10270000FFFFFFFFFFFFFFFFFFFFFF0FFFFF0000C7
:102710000FFFFC00000FFFF03FFF0FFFF0FFFFFF78
:10272000FFF0FFFFFFFFF03FFF0FFFFC00000FFF78
:10273000FF00000FFFFFFFFF0FFFFFFFFFFFFFFF87
:10274000FFFFFFFFFFFFFFFFFFFFFFFF0FFFFFFF89
:10275000F00FFFFFFF000FFFFFC00F0FFFF000FFA4
:10276000FFFFF03FFFFFFFF000FFFFFFFFC00F0F75
:10277000FFFFFF000FFFFFFFF00FFFFFFFFF0FFF47
:10278000FFFFFFFFFFFFFFFFFFFFFFFFFFFFFFFF59
:10279000FFFF0FFFFFFC000FFFF000000FFFF00F27
:1027A000FF0FFFFC00FF0FFFFFF003FFFFFFFF0322
:1027B000FFFFFFF003FFFFFC00FF0FFFF00FFF0F15
:1027C000FFF000000FFFFFFC000FFFFFFFFF0FFFF8
:1027D000FFFFFFFFFFF0FFFF0FFFF03FFC0FFFF0D9
:1027E0000FF00FFFF0C3C30FFFFFF00FFFFFFFFC61
:1027F0003FFFFFFFF00FFFFFF0C3C30FFFF00FF02D
:102800000FFFF03FFC0FFFF0FFFF0FFFFFFFFFFF89
:10281000FFFFFFFFFFFFFFFFFFFFFFFFFFFFFFFFC8
:10282000FFFFFF0FFFFFFFFC0FFFF0FFF00FFFF0B8
:10283000FF030FFFF0000FFFFFF0000FFFFFF0FF9F
:10284000030FFFF0FFF00FFFFFFFFC0FFFFFFFFF85
:102850000FFFFFFFFFFFFFFFFFFFFFFFFFFFFFFF78
:10286000FFFFFFFFFFFFFFFFFFFFFFF03FF00FFF46
:10287000F00FF00FFFF0C3FF0FFFF0F03F0FFFF07E
:10288000FC0F0FFFF0FFC30FFFF00FF00FFFF00F73
:10289000FC0FFFFFFFFFFFFFFFFFFFFFFFFFFFFF3B
:1028A000FFFFFFFFFFFFFFFFFFFFFFFFFFFFFFFF38
:1028B000FFFFFFFFFFFFFFFFFFFFFFFFFFFFFFFC2B
:1028C0000000000FFC0000000FFC3FFFFF0FFC3F6B
:1028D000FFFF0FFFFFFFFFFFFFFFFFFFFFFFFFFFF8
:1028E000FFFFFFFFFFFFFFFFFFFFFFFFFFFFFFFFF8
:1028F000FFFFFFFFFFFFFFFFFFFFF0FFFFFFFC00F9
:10290000FFFFFFC00FFFFFFC03FFFFFFC03FFFFF04
:10291000F003FFFFFF003FFFFFFF0FFFFFFFFFFF81
:10292000FFFFFFFFFFFFFFFFFFFFFFFFFFFFFFFFB7
:10293000FFFFFFFFFFFFFFFFFFFFFFFFFFFFFFFFA7
:10294000FFFC3FFFFF0FFC3FFFFF0FFC0000000FED
:10295000FC0000000FFFFFFFFFFFFFFFFFFFFFFF77
:10296000FFFFFFFFFFFFFFFFFFFFFFFFFFFFFFFF77
:10297000FFFFFFFFFFFFFFFFFFFFFFFFFFFFFFFF67
:10298000C3FFFFFFFFF0FFFFFFFFFC3FFFFFFFFF65
:102990000FFFFFFFFFC3FFFFFFFF0FFFFFFFFC3F26
:1029A000FFFFFFF0FFFFFFFFC3FFFFFFFFFFFFFF82
:1029B000FFFFFFFFFFFFFFFFFF0FFFFFFFFF0FFF07
:1029C000FFFFFF0FFFFFFFFF0FFFFFFFFF0FFFFFE7
:1029D000FFFF0FFFFFFFFF0FFFFFFFFF0FFFFFFFD7
:1029E000FF0FFFFFFFFF0FFFFFFFFF0FFFFFFFFFC7
:1029F0000FFFFFFFFF0FFFFFFFFF0FFFFFFFFFFFB7
:102A0000FFFFFFFFFFFFFFFFFFFFFFFFFFFFFFFFD6
:102A1000FFFFFFFFFFFFFFFFFFFFFFFFF3FFFFFFD2
:102A2000FFCFFFFFFFFFCFFFFFFFFF3FFFFFFFFFD6
:102A3000FFFFFFFFFFFFFFFFFFFFFFFFFFFFFFFFA6
:102A4000FFFFFFFFFFFFFFFFFFFFFFFFFFFFFFFF96
:102A5000FC0FFFFFFFF003CFFFFFF0C0C3FFFFF04D
:102A6000F0C3FFFFF0F0C3FFFFFC30C3FFFFF00037
:102A700003FFFFF0000FFFFFF0FFFFFFFFFFFFFF6F
:102A8000FFFFFFFFFFFFFFFFFFFFFFFFFFFFFFFF56
:102A9000FFF0FFFFC3FFF0000003FFF0000003FFA3
:102AA000FC3F0FFFFFF0FFC3FFFFF0FFC3FFFFF08E
:102AB000FFC3FFFFF0FFC3FFFFFC3F0FFFFFFC0062
:102AC0000FFFFFFFC0FFFFFFFFFFFFFFFFFFFFFF45
:102AD000FFFFFFFFFFFFFFFFFFFFFFFFFF00FFFF05
:102AE000FFFC000FFFFFF03F0FFFFFF0FFC3FFFFF2
:102AF000F0FFC3FFFFF0FFC3FFFFF0FFC3FFFFF0D6
:102B0000FFCFFFFFFC3C03FFFFFC3C03FFFFFFFF89
:102B1000FFFFFFFFFFFFFFFFFFFFFFFFFFFFFFFFC5
:102B2000FFFFFF00FFFFFFFC000FFFFFFC3F0FFF59
:102B3000FFF0FFC3FFFFF0FFC3FFFFF0FFC3FFFF86
:102B4000F0FFC3FFFFFC3F0FC3FFF0000003FFF0E7
:102B5000000003FFF0FFFFFFFFFFFFFFFFFFFFFF8E
:102B6000FFFFFFFFFFFFFFFFFFC0FFFFFFFC000FA6
:102B7000FFFFFC300FFFFFF0F0C3FFFFF0F0C3FFDB
:102B8000FFF0F0C3FFFFF0F0C3FFFFF0F00FFFFF17
:102B9000FC300FFFFFFC30FFFFFFFFFFFFFFFFFFD9
:102BA000FFFFFFFFFFFFFFFFFFFFFFFFFFFFFFFF35
:102BB000FFFFFFF0FFC3FFFFF0FFC3FFFFF00000C8
:102BC0000FFFF0000003FFF0FFC3C3FFF0FFC3C31C
:102BD000FFF0FFC3C3FFF0FFC3C3FFFFFFFFC3FF4F
:102BE000FFFFFFFFFFFFFFFFFFFFFFFFFFFFFFFFF5
:102BF000FFFFFFFFFFC0FFFFFFFC000FFFF0FC3FE8
:102C00000FFFF0F0FFC3FFF0F0FFC3FFF0F0FFC3D2
:102C1000FFF0F0FFC3FFF03C3F0FFFFC000003FF9D
:102C2000FF000003FFFFFFFFC3FFFFFFFFFFFFFFEA
:102C3000FFFFFFFFFFFFFFFFFFFFF0FFFFC3FFF0FE
:102C4000000003FFF0000003FFF0FF0FFFFFFFFF96
:102C5000C3FFFFFFFFC3FFFFF0FFC3FFFFF0000351
:102C6000FFFFF0000FFFFFF0FFFFFFFFFFFFFFFF81
:102C7000FFFFFFFFFFFFFFFFFFFFFFFFFFFFFFFF64
:102C8000FFFFFFFFFFF0FFC3FFFFF0FFC3FFFFF0F9
:102C9000FFC3FFFFF00003C3FFF00003C3FFF0FF1B
:102CA000FFFFFFF0FFFFFFFFF0FFFFFFFFFFFFFF52
:102CB000FFFFFFFFFFFFFFFFFFFFFFFFFFFFFFFF24
:102CC000FFFFFFFFFFFFFFFFFFFFF0FFFFFFFFF032
:102CD000FFFFC3FFF0FFFFC3FFF0FFFFC3FFF0FFE5
:102CE000FFC3C3F0FFFFC3C3FC000003FFFF0000EE
:102CF00003FFFFFFFFFFFFFFFFFFFFFFFFFFFFFFE0
:102D0000FFFFFFFFFFFFFFFFFFFFFFFFF0FFFFC31E
:102D1000FFF0000003FFF0000003FFFFF0FFFFFFE4
:102D2000FFC003FFFFF00F03FFFFF03FC3FFFFF003
:102D3000FFC3FFFFF0FFC3FFFFF0FFFFFFFFFFFF39
:102D4000FFFFFFFFFFFFFFFFFFFFFFFFFFFFFFFF93
:102D5000FFFFFFFFFFFFFFF0FFFFC3FFF0FFFFC319
:102D6000FFF0FFFFC3FFF0000003FFF0000003FFD0
:102D7000F0FFFFFFFFF0FFFFFFFFF0FFFFFFFFFF90
:102D8000FFFFFFFFFFFFFFFFFFFFFFFFFFFFFFFF53
:102D9000FFFFFFF0FFC3FFFFF00003FFFFF00003A2
:102DA000FFFFF0FFC3FFFFFFFFC3FFFFF00003FFC4
:102DB000FFF0000FFFFFF0FFC3FFFFFFFFC3FFFFA8
:102DC000F00003FFFFF0000FFFFFF0FFFFFFFFFF2A
:102DD000FFFFFFFFFFFFFFFFFFFFFFFFFFFFF0FF12
:102DE000C3FFFFF00003FFFFF00003FFFFF0FF0F42
:102DF000FFFFFFFFC3FFFFFFFFC3FFFFF0FFC3FFA6
:102E0000FFF00003FFFFF0000FFFFFF0FFFFFFFFE9
:102E1000FFFFFFFFFFFFFFFFFFFFFFFFFFFFFFFFC2
:102E2000FFFFFFFFFFC0FFFFFFFC000FFFFFFC3FA6
:102E30000FFFFFF0FFC3FFFFF0FFC3FFFFF0FFC373
:102E4000FFFFF0FFC3FFFFFC3F0FFFFFFC000FFF82
:102E5000FFFFC0FFFFFFFFFFFFFFFFFFFFFFFFFFC1
:102E6000FFFFFFFFF0FFFFC3FFF0000003FFF000D4
:102E70000003FFF0FC3F0FFFF0F0FFC3FFFFF0FF88
:102E8000C3FFFFF0FFC3FFFFF0FFC3FFFFFC3F0FD7
:102E9000FFFFFC000FFFFFFFC0FFFFFFFFFFFFFF73
:102EA000FFFFFFFFFFFFFFFFFFFFFFFFFFFFFFFF32
:102EB000FFC0FFFFFFFC000FFFFFFC3F0FFFFFF015
:102EC000FFC3FFFFF0FFC3FFFFF0FFC3FFF0F0FF02
:102ED000C3FFF0FC3F0FFFF0000003FFF000000312
:102EE000FFF0FFFFC3FFFFFFFFFFFFFFFFFFFFFF3D
:102EF000FFFFFFFFFFFFF0FFC3FFFFF0FFC3FFFF78
:102F0000F00003FFFFF00003FFFFF0FC3FFFFFF0C6
:102F1000FF0FFFFFF0FFC3FFFFF0FFC3FFFFFFFF47
:102F200003FFFFFFFF0FFFFFFFFFFFFFFFFFFFFF9D
:102F3000FFFFFFFFFFFFFFFFFFFFFFFFFFFFFFFFA1
:102F4000FFF03C0FFFFFF0300FFFFFF0F0C3FFFF7B
:102F5000F0F0C3FFFFF0C3C3FFFFF0C3C3FFFFFCEC
:102F60000303FFFFFC0F03FFFFFFFFFFFFFFFFFF58
:102F7000FFFFFFFFFFFFFFFFFFFFFFFFFFFFFFFF61
:102F8000FFFFFFFFC3FFFFFFFFC3FFFFFC00000FBA
:102F9000FFF000000FFFF0FFC3FFFFF0FFC3FFFFD4
:102FA000F0FFC3FFFFF0FFC3FFFFFC3FC3FFFFFCC9
:102FB0003FFFFFFFFFFFFFFFFFFFFFFFFFFFFFFFE1
:102FC000FFFFFFFFFFFFFFFFFFFFC3FFFFFC00034B
:102FD000FFFFF00003FFFFF0FFFFFFFFF0FFFFFF29
:102FE000FFF0FFFFFFFFFC3FC3FFFFF00003FFFF09
:102FF000F00003FFFFF0FFFFFFFFFFFFFFFFFFFFFA
:10300000FFFFFFFFFFFFFFFFFFFFFFC3FFFFFFFF0C
:1030100003FFFFFFF003FFFFFF00C3FFFFF00FFF01
:10302000FFFFF0FFFFFFFFF00FFFFFFFFF00C3FFF9
:10303000FFFFF003FFFFFFFF03FFFFFFFFC3FFFFE3
:10304000FFFFFFFFFFFFFFFFFFFFFFFFFFFFFFFF90
:10305000FFC3FFFFFFF003FFFFF00003FFFFF00FD0
:10306000C3FFFFFF03FFFFFFFFF03FFFFFFF03FF73
:10307000FFFFF00FC3FFFFF00003FFFFFFF003FFB0
:10308000FFFFFFC3FFFFFFFFFFFFFFFFFFFFFFFF8C
:10309000FFFFFFFFFFFFFFFFFFFFF0FFC3FFFFF09A
:1030A000FFC3FFFFF03F03FFFFF00C03FFFFFFC074
:1030B000FFFFFFFFC0FFFFFFF00C03FFFFF03F0328
:1030C000FFFFF0FFC3FFFFF0FFC3FFFFFFFFFFFFA6
:1030D000FFFFFFFFFFFFFFFFFFFFF0FFFFC3FFF05A
:1030E000FFFF03FFF0FFF003FFF03F00C3FFF0001E
:1030F0000FFFFFF0C03FFFFFF0FC0FFFFFFFFF00DF
:10310000C3FFFFFFF003FFFFFFFF03FFFFFFFFC34E
:10311000FFFFFFFFFFFFFFFFFFFFFFFFFFFFFFFFBF
:10312000FFFFFFFFFFFFFFFFFFFFFFF0FF03FFFFBA
:10313000F03F03FFFFF00FC3FFFFF0C3C3FFFFF03B
:10314000F0C3FFFFF0FC03FFFFF03F03FFFFF03F82
:10315000C3FFFFFFFFFFFFFFFFFFFFFFFFFFFFFFBB
:10316000FFFFFFFFFFFFFFFFFFFFFFFFFFFFFFFF6F
:10317000FFFFFFFFFFFFFFF3FFFFFFFFC0FFFFFFAA
:103180000000000FFC000C0003FC3FFFFFC3FC3FEE
:10319000FFFFC3FFFFFFFFFFFFFFFFFFFFFFFFFF7B
:1031A000FFFFFFFFFFFFFFFFFFFFFFFFFFFFFFFF2F
:1031B000FFFFFFFFFFFFFFFFFFFFFFFFFFFFFFFF1F
:1031C000FFFFFFFFFFFC00000003FC00000003FF07
:1031D000FFFFFFFFFFFFFFFFFFFFFFFFFFFFFFFFFF
:1031E000FFFFFFFFFFFFFFFFFFFFFFFFFFFFFFFFEF
:1031F000FFFFFFFFFFFFFFFFFFFFFFFFFC3FFFFFA2
:10320000C3FC3FFFFFC3FC000C0003FF0000000FE6
:10321000FFFFC0FFFFFFFFF3FFFFFFFFFFFFFFFF09
:10322000FFFFFFFFFFFFFFFFFFFFFFFFFFFFFFFFAE
:10323000FFFFFFFFFFFFFFFFFFFFFFFFFFFFFFFCA1
:103240003FFFFFFFFC3FFFFFFFFF0FFFFFFFFF0FF1
:10325000FFFFFFFC0FFFFFFFF03FFFFFFFF0FFFF4F
:10326000FFFFF0FFFFFFFFF03FFFFFFFFC3FFFFF0F
:10327000FFFFFFFFFFFFFFFFFFFFFFFFFFFFFFFF5E
:10328000FFFFFFFFFFFFFFFFFFFFFFFFFFFFFFFF4E
:10329000FFFFFFFFFFFFFFFFFFFFFFFFFFFFFFFF3E
:1032A000FFFFFFFFFFFFFFFFFFFFFFFFFFFFFFFF2E
:1032B000FFFFFFFFFFFFCC0003FFCC0003FFFFFF7A
:1032C000FFFFFFFFFFFFFFFFFFFFFFFFFFFFFFFF0E
:1032D000FFFFFFFFFFFFFFFFFFFFFFFFFFFFFFFFFE
:1032E0000FFFFFC00FFFFFFF0FFFFFFFFFFFFFFFFD
:1032F0000FFFFFC00FFFFFFF0FFFFFFFFFFFFFFFED
:10330000FFFFFFFFFFFFFF33FFFF0003FFFF000092
:1033100003FFFF3003FF0003FFFF000003FFFF3048
:1033200003FFFF33FFFFFFFFFFFFFFFFFFFFFFFF75
:10333000FFFFC0FC0FFFC0F003FFCFC0F3FC0FC3C3
:10334000F0FFCF03F3FFC00F03FFF03F03FFFFFFCA
:10335000FFFFFFFFFFFFFFFFFFFFFFFFFFFFFF3F3D
:103360000FFFFF0CF3FFFFCCF3FFFFC30FFFF0C312
:10337000FFFFCF33FFFFCF30FFFFF0FCFFFFFFFF6A
:10338000FFFFFFFFFFFFFFFFFFFFF0FFFFFFC0306A
:103390003FFFCF000FFFCC0FCFFFF0FFCFFFC03FAD
:1033A000CFFFCF3FCFFFFFFFFFFFFFFFFFFFFFFF7D
:1033B000FFFFFFFFFFFFFFFFFFFFFFFFFFFFFFFF1D
:1033C000FFFFFFFF0FFFFFC00FFFFFFF0FFFFFFF1C
:1033D000FFFFFFFFFFFFFFFFFFFFFFFFFFFFFFFFFD
:1033E000FFFFFFFFFFFFFFFFFFFFF000FFFFC00039
:1033F0003FFC03FC03FC3FFFC3FFFFFFFFFFFFFF9A
:10340000FFFFFFFFFFFFFFFFFFFFFFFFFFFFFFFFCC
:10341000FFFC3FFFC3FC03FC03FFC0003FFFF000C5
:10342000FFFFFFFFFFFFFFFFFFFFFFFFFFFFFFFFAC
:10343000FFFFFFFFFFFFFFFFFFFFFFFC3FFFFF0C52
:103440003FFFFF003FFFFFF003FFFFF003FFFF0020
:103450003FFFFF0C3FFFFFFC3FFFFFFFFFFFFFFFB2
:10346000FFFFFFFFFFFFFFCFFFFFFFCFFFFFFFCFFC
:10347000FFFFF0003FFFFFCFFFFFFFCFFFFFFFCFBA
:10348000FFFFFFFFFFFFFFFFFFFFFFFFFFFFFFFF4C
:10349000FFFFFFFFFFFFFFFFFFF03FFFFFFF03FF07
:1034A000FFFFF3FFFFFFFFFFFFFFFFFFFFFFFFFF38
:1034B000FFFFFFFFFFFFFFFFFFFFFFFFFFFFFFCF4C
:1034C000FFFFFFCFFFFFFFCFFFFFFFCFFFFFFFCFCC
:1034D000FFFFFFCFFFFFFFCFFFFFFFFFFFFFFFFF5C
:1034E000FFFFFFFFFFFFFFFFFFFFFFFFFFFFFFFFEC
:1034F000FFFFC3FFFFFFC3FFFFFFFFFFFFFFFFFF54
:10350000FFFFFFFFFFFFFFFFFFFFFFFFFFFFFFFFCB
:10351000FFFFFFFFFFFC3FFFFFFC03FFFFFFC03F7C
:10352000FFFFFC0FFFFFFFC0FFFFFFF00FFFFFFFDC
:1035300000FFFFFFF0FFFFFFFFFFFFFFFFFFFFFFA9
:10354000FFFFFC003FFFF0000FFFC3FFC3FFCFFFF3
:10355000F3FFC3FFC3FFF0000FFFFC003FFFFFFFBF
:10356000FFFFFFFFFFFFFFFFFFFFFFFFFFFFCFFF9B
:10357000CFFFCFFFCFFFCFFFCFFFC00003FFC000C3
:1035800003FFCFFFFFFFCFFFFFFFCFFFFFFFFFFFD7
:10359000FFFFFFFFFFFFFFFFFFFFC3FC3FFFC0FC7C
:1035A0000FFFCC3FC3FFCF0FF3FFCFC3F3FFCFF02D
:1035B00003FFCFFC0FFFFFFFFFFFFFFFFFFFFFFF3A
:1035C000FFFFF3FFCFFFC3FFC3FFCFF3F3FFCFF343
:1035D000F3FFCFF3F3FFCFC0F3FFC00003FFF00F03
:1035E0000FFFFFFFFFFFFFFFFFFFFFFFFFFFFFFFDB
:1035F000FFFFFC3FFFFFFC03FFFFCCF03FFFCCFFD2
:1036000003FFC00003FFC00003FFCCFFFFFFFFFF6D
:10361000FFFFFFFFFFFFFFFFFFFFFFFFFFFFF3FFC6
:10362000FFFFCFC003FFCFF003FFCFF3F3FFCFF3D4
:10363000F3FFC003F3FFF00FF3FFFFFFFFFFFFFFF8
:10364000FFFFFFFFFFFFFFFFFFFFFC00FFFFF0009A
:103650003FFFC3CF0FFFCFF3C3FFCFF3F3FFC00391
:10366000F3FFF00FF3FFFFFFFFFFFFFFFFFFFFFF81
:10367000FFFFFFFFFFFFFFFFC3FFFFFFF3FFFFFFA2
:10368000F3FFC0FFF3FFC000F3FFFF0003FFFFFFE6
:1036900003FFFFFFFFFFFFFFFFFFFFFFFFFFFFFF36
:1036A000FFFFF00C0FFFC00003FFCFF3F3FFCFF3DA
:1036B000F3FFCFF3F3FFC00003FFF00C0FFFFFFF9A
:1036C000FFFFFFFFFFFFFFFFFFFFFFFFFFFFCFF049
:1036D0000FFFCFC003FFCFCFF3FFC3CFF3FFF0F354
:1036E000C3FFF0000FFFFF003FFFFFFFFFFFFFFFE3
:1036F000FFFFFFFFFFFFFFFFFFFFFFFFFFFFFFFFDA
:10370000FFFFC3F0FFFFC3F0FFFFFFFFFFFFFFFF5F
:10371000FFFFFFFFFFFFFFFFFFFFFFFFFFFFFFFFB9
:10372000FFFFFFFFFFFFFFFFFFFFFFFFFFFC3FFF6C
:10373000FFFFC3FFFFFFF3F0FFFFFFF0FFFFFFFFFF
:10374000FFFFFFFFFFFFFFFFFFFFFFFFFFFFFFCFB9
:10375000FFFFFFCFFFFFFF33FFFFFF33FFFFFCFC47
:10376000FFFFF3FF3FFFF3FF3FFFCFFFCFFFCFFF91
:10377000CFFFFFFFFFFFFFFFFFFFFFFFFFFFFF3355
:10378000FFFFFF33FFFFFF33FFFFFF33FFFFFF3379
:10379000FFFFFF33FFFFFF33FFFFFFFFFFFFFFFFD1
:1037A000FFFFFFFFFFFFCFFFCFFFCFFFCFFFF3FFF5
:1037B0003FFFF3FF3FFFFCFCFFFFFF33FFFFFF3343
:1037C000FFFFFFCFFFFFFFCFFFFFFFFFFFFFFFFF69
:1037D000FFFFFFFFFFFFFFFC3FFFFFFC0FFFCC3FA2
:1037E000CFFFCC0FCFFFFFCFCFFFFFC00FFFFFF00A
:1037F0003FFFFFFFFFFFFFFFFFFFFFFFFFFFFFFF99
:10380000FFFFF0003FFFCFFFCFFF3F0FF3FF3CF381
:10381000F3FF3CF3F3FFCC000FFFFFFFFFFFFFFFC1
:10382000FFFFFFFFFFFFFFFFFFFFCFFFFFFFC0FF17
:10383000CFFFC003CFFFCF000FFFFF3F0FFFFF3FC2
:103840000FFFCF000FFFC003FFFFC0FFFFFFCFFF41
:10385000FFFFFFFFFFFFCFFFCFFFC0000FFFC00044
:103860000FFFCFCFCFFFCFCFCFFFCFCFCFFFC00046
:103870000FFFF0303FFFFFFFFFFFFFFFFFFFFFFFE6
:10388000FFFFFC00FFFFF0003FFFC3FF0FFFCFFF74
:10389000CFFFCFFFCFFFCFFFCFFFCFFFCFFFF3FF94
:1038A0003FFFFCFC0FFFFFFFFFFFFFFFFFFFCFFF0E
:1038B000CFFFC0000FFFC0000FFFCFFFCFFFCFFF34
:1038C000CFFFCFFFCFFFC3FF0FFFF0003FFFFC0094
:1038D000FFFFFFFFFFFFFFFFFFFFCFFFCFFFC00096
:1038E0000FFFC0000FFFCFCFCFFFCFCFCFFFCF0352
:1038F000CFFFCFFFCFFFC0FC0FFFFFFFFFFFFFFF9A
:10390000FFFFFFFFFFFFCFFFCFFFC0000FFFC00093
:103910000FFFCFCFCFFFCFCFCFFFFF03CFFFFFFFF3
:10392000CFFFFFFC0FFFFFFFFFFFFFFFFFFFFFFFCA
:10393000FFFFFC00FFFFF0003FFFC3FF0FFFCFFFC3
:10394000CFFFCF3FCFFFCF3FCFFFC03F3FFFC03CB8
:103950000FFFFF3FFFFFFFFFFFFFFFFFFFFFCFFF57
:10396000CFFFC0000FFFC0000FFFCFCFCFFFFFCFB3
:10397000FFFFCFCFCFFFC0000FFFC0000FFFCFFF73
:10398000CFFFFFFFFFFFFFFFFFFFFFFFFFFFCFFFA7
:10399000CFFFCFFFCFFFCFFFCFFFC0000FFFC00093
:1039A0000FFFCFFFCFFFCFFFCFFFCFFFCFFFFFFF37
:1039B000FFFFFFFFFFFFF03FFFFFC03FFFFFCFFF15
:1039C000CFFFCFFFCFFFCFFFCFFFC0000FFFF00033
:1039D0000FFFFFFFCFFFFFFFCFFFFFFFFFFFFFFF47
:1039E000FFFFCFFFCFFFC0000FFFC0000FFFCF0FC3
:1039F000CFFFFF03FFFFFC30CFFFC0FC0FFFC3FF73
:103A00000FFFCFFFCFFFFFFFFFFFFFFFFFFFCFFF46
:103A1000CFFFCFFFCFFFC0000FFFC0000FFFCFFFD2
:103A2000CFFFCFFFCFFFCFFFFFFFCFFFFFFFC03F95
:103A3000FFFFFFFFFFFFCFFFCFFFC0000FFFC00062
:103A40000FFFCFF0FFFFCF03FFFFFC3FFFFFCF03D0
:103A5000FFFFCFF0FFFFC0000FFFC0000FFFCFFF41
:103A6000CFFFFFFFFFFFCFFFCFFFC0000FFFC00062
:103A70000FFFCFF0FFFFFF03FFFFFC3FCFFFC000B2
:103A80000FFFC0000FFFFFFFCFFFFFFFFFFFFFFF94
:103A9000FFFFFC00FFFFF0003FFFC3FF0FFFCFFF62
:103AA000CFFFCFFFCFFFCFFFCFFFC3FF0FFFF00050
:103AB0003FFFFC00FFFFFFFFFFFFFFFFFFFFCFFF08
:103AC000CFFFC0000FFFC0000FFFCF3FCFFFCF3FA2
:103AD000CFFFCF3FCFFFFF000FFFFFC03FFFFFFF34
:103AE000FFFFFFFFFFFFFFFFFFFFFC00FFFFF000F6
:103AF0003FFCC3FF0FFC0FFFCFFC0FFFCFFCCFFF3E
:103B0000CFFCC3FF0FFC30003FFF3C00FFFFFFFF77
:103B1000FFFFFFFFFFFFCFFFCFFFC0000FFFC00081
:103B20000FFFCFCFCFFFCFCFCFFFFF0FCFFFF030B3
:103B30000FFFC0F03FFFCFFFFFFFCFFFFFFFFFFFF3
:103B4000FFFFFFFFFFFFC0F03FFFC0C00FFFCFC36D
:103B5000CFFFCFCFCFFFCF0FCFFFC00C0FFFF03C79
:103B60000FFFFFFFFFFFFFFFFFFFFFFFFFFFFFF064
:103B70000FFFCFFFCFFFCFFFCFFFC0000FFFC00071
:103B80000FFFCFFFCFFFCFFFCFFFFFF00FFFFFFFF4
:103B9000FFFFFFFFFFFFFFFFFFFFFFFFCFFFF00073
:103BA0000FFFF0000FFFCFFFCFFFCFFFFFFFCFFFD3
:103BB000CFFFF0000FFFF0000FFFFFFFCFFFFFFF71
:103BC000FFFFFFFFFFFFFFFFCFFFFFFC0FFFFF0027
:103BD0000FFFC003CFFFC3FFFFFFC003CFFFFF00F6
:103BE0000FFFFFFC0FFFFFFFCFFFFFFFFFFFFFFFF8
:103BF000CFFFFFC00FFFC0000FFFC0FFCFFFF003DC
:103C0000CFFFFFC0FFFFF003CFFFC0FFCFFFC0001B
:103C10000FFFFFC00FFFFFFFCFFFFFFFFFFFCFFF33
:103C2000CFFFC3FF0FFFC0FC0FFFCC00CFFFFF0390
:103C3000FFFFCC00CFFFC0FC0FFFC3FF0FFFCFFF84
:103C4000CFFFFFFFFFFFFFFFFFFFFFFFCFFFFFFFE4
:103C50000FFFCFFC0FFFCFF0CFFFC003FFFFC0036C
:103C6000FFFFCFF0CFFFCFFC0FFFFFFF0FFFFFFFE6
:103C7000CFFFFFFFFFFFFFFFFFFFC3FC0FFFC0FFF2
:103C8000CFFFCC3FCFFFCF03CFFFCFF0CFFFCFFC95
:103C90000FFFC0FF0FFFFFFFFFFFFFFFFFFFFFFF53
:103CA000FFFFFFFFFFFFFFFFFFFFFFFFFFFFFFFF24
:103CB000FFFC000003FC000003FCFFFFF3FCFFFF20
:103CC000F3FFFFFFFFFFFFFFFFFFFFFFFFFFFFFF10
:103CD000FFFFFFFFF0FFFFFF00FFFFF00FFFFFC040
:103CE000FFFFFC0FFFFFC03FFFFC03FFFFFC3FFF98
:103CF000FFFFFFFFFFFFFFFFFFFFFFFFFFFFFFFFD4
:103D0000FFFCFFFFF3FCFFFFF3FC000003FC0000DF
:103D100003FFFFFFFFFFFFFFFFFFFFFFFFFFFFFFAF
:103D2000FFFFFFFFFFFFFFFFFFFFFFF0FFFFFFFFB2
:103D30003FFFFFFFC3FFFFFFFCFFFFFFC3FFFFFFCE
:103D40003FFFFFF0FFFFFFFFFFFFFFFFFF3FFFFF12
:103D5000FF3FFFFFFF3FFFFFFF3FFFFFFF3FFFFF73
:103D6000FF3FFFFFFF3FFFFFFF3FFFFFFF3FFFFF63
:103D7000FF3FFFFFFF3FFFFFFFFFFFFFFFFFFFFFD3
:103D8000FFFFFFFFFFFFFFFFFFFFFFFFFCFFFFFF46
:103D9000F3FFFFFFCFFFFFFFFFFFFFFFFFFFFFFF6F
:103DA000FFFFFFFFFFFFFFFFFFFFFFFFFFFFF0FF32
:103DB000FFFFC03CFFFFCF3CFFFFCF3CFFFFF33CCA
:103DC000FFFFC000FFFFC003FFFFCFFFFFFFFFFFAC
:103DD000FFFFFFFFFFFFCFFFF3FFC00003FFC000A7
:103DE00003FFF3F3FFFFCFFCFFFFCFFCFFFFC3F0A8
:103DF000FFFFF003FFFFFC0FFFFFFFFFFFFFFFFFD1
:103E0000FFFFFC0FFFFFF003FFFFC3F0FFFFCFFC3E
:103E1000FFFFCFFCFFFFCFFCFFFFC3F3FFFFF0C0AE
:103E2000FFFFFFFFFFFFFFFFFFFFFFFFFFFFFC0F95
:103E3000FFFFF003FFFFC3F0FFFFCFFCFFFFCFFC4E
:103E4000FFFFF3F3F3FFC00003FFC00003FFCFFF4A
:103E5000FFFFFFFFFFFFFFFFFFFFFC0FFFFFF00370
:103E6000FFFFC330FFFFCF3CFFFFCF3CFFFFCF3052
:103E7000FFFFC303FFFFF30FFFFFFFFFFFFFFFFF86
:103E8000FFFFFFFFFFFFFFFFFFFFCFFCFFFFCFFCA8
:103E9000FFFFC0000FFFC00003FFCFFCF3FFCFFC0C
:103EA000F3FFCFFCF3FFFFFFF3FFFFFFF3FFFFFF85
:103EB000FFFFFC0FFFFFF003FFF3C3F0FFF3CFFCA6
:103EC000FFF3CFFCFFF3F3F3FFF00000FFFC000073
:103ED000FFFFFFFCFFFFFFFFFFFFFFFFFFFFCFFF25
:103EE000F3FFC00003FFC00003FFCFF3FFFFFFFCA1
:103EF000FFFFCFFCFFFFC000FFFFC003FFFFCFFFAE
:103F0000FFFFFFFFFFFFFFFFFFFFFFFFFFFFCFFFF1
:103F1000FFFFCFFCFFFFCFFCFFFFC000C3FFC000CF
:103F2000C3FFCFFFFFFFCFFFFFFFCFFFFFFFFFFF6D
:103F3000FFFFFFFFFFFFFFFFFFF3FFFCFFF3FFFCAF
:103F4000FFF3FFFCFFF3FFFCC3F00000C3FC000025
:103F5000FFFFFFFFFFFFFFFFFFFFFFFFFFFFFFFF71
:103F6000FFFFCFFFF3FFC00003FFC00003FFFF0F01
:103F7000FFFFCC00FFFFC0F0FFFFC3FCFFFFCFFC43
:103F8000FFFFCFFFFFFFFFFFFFFFFFFFFFFFCFFFA1
:103F9000FFFFCFFFF3FFCFFFF3FFC00003FFC00021
:103FA00003FFCFFFFFFFCFFFFFFFCFFFFFFFFFFFAD
:103FB000FFFFFFFFFFFFFFFFFFFFCFFCFFFFC00082
:103FC000FFFFC000FFFFFFFCFFFFC000FFFFC000BE
:103FD000FFFFFFFCFFFFC000FFFFC003FFFFCFFF9D
:103FE000FFFFFFFFFFFFCFFCFFFFC000FFFFC00090
:103FF000FFFFCFF3FFFFFFFCFFFFCFFCFFFFC00081
:10400000FFFFC003FFFFCFFFFFFFFFFFFFFFFFFF2B
:10401000FFFFFC0FFFFFF003FFFFC3F0FFFFCFFC2C
:10402000FFFFCFFCFFFFCFFCFFFFC3F0FFFFF0035C
:10403000FFFFFC0FFFFFFFFFFFFFFFFFFFF3FFFC92
:10404000FFF00000FFF00000FFF3F3F3FFF3CFFCFD
:10405000FFFFCFFCFFFFC3F0FFFFF003FFFFFC0FEC
:10406000FFFFFFFFFFFFFFFFFFFFFC0FFFFFF0035E
:10407000FFFFC3F0FFFFCFFCFFF3CFFCFFF3F3F331
:10408000FFF00000FFF00000FFF3FFFCFFFFFFFF69
:10409000FFFFFFFFFFFFCFFCFFFFCFFCFFFFC000D4
:1040A000FFFFC000FFFFCFF3FFFFCFFCFFFFCFFC00
:1040B000FFFFFFF0FFFFFFF3FFFFFFFFFFFFFFFF2B
:1040C000FFFFC3C3FFFFC300FFFFCF0CFFFFCF0CF9
:1040D000FFFFCC3CFFFFC030FFFFF0F0FFFFFFFF12
:1040E000FFFFFFFFFFFFFFFFFFFFFFFFFFFFFFFCE3
:1040F000FFFFFFFCFFFFF00003FFC00003FFCFFC4A
:10410000FFFFCFFCFFFFCFFCFFFFF3FFFFFFFFFF31
:10411000FFFFFFFFFFFFFFFFFFFFFFFCFFFFF000C0
:10412000FFFFC000FFFFCFFFFFFFCFFFFFFFF3FC4C
:10413000FFFFC000FFFFC000FFFFCFFFFFFFFFFF3B
:10414000FFFFFFFFFFFFFFFCFFFFFFC0FFFFFC00C3
:10415000FFFFC03CFFFFC3FFFFFFC03CFFFFFC00B1
:10416000FFFFFFC0FFFFFFFCFFFFFFFFFFFFFFFCA4
:10417000FFFFFF00FFFFC000FFFFC0FCFFFFF03F9D
:10418000FFFFFF0FFFFFF03FFFFFC0FCFFFFC0007E
:10419000FFFFFF00FFFFFFFCFFFFFFFFFFFFCFFC64
:1041A000FFFFCFFCFFFFC3F0FFFFC000FFFFFC0FCE
:1041B000FFFFC000FFFFC3F0FFFFCFFCFFFFCFFCFE
:1041C000FFFFFFFFFFFFFFFFFFFFFFFCFFF3FFF01D
:1041D000FFF3FF00FFF0F00CFFF003FFFFF300FF21
:1041E000FFFFF00CFFFFFF00FFFFFFF0FFFFFFFCF2
:1041F000FFFFFFFFFFFFFFFFFFFFC3F0FFFFC0FC5C
:10420000FFFFCC3CFFFFCF3CFFFFCF0CFFFFCFC039
:10421000FFFFC3F0FFFFFFFFFFFFFFFFFFFFFFFFF9
:10422000FFFFFFFFFFFFFFFFFFFFFF3FFFFF00005C
:104230000FFC00C003FCFFFFF3FFFFFFFFFFFFFFCA
:10424000FFFFFFFFFFFFFFFFFFFFFFFFFFFFFFFF7E
:10425000FFFFFFFFFFFFFFFFFFFFFFFFFFFC00006F
:1042600003FC000003FFFFFFFFFFFFFFFFFFFFFF57
:10427000FFFFFFFFFFFFFFFFFFFFFFFFFFFFFFFF4E
:10428000FFFFFFFFFFFCFFFFF3FC00C003FF000088
:104290000FFFFF3FFFFFFFFFFFFFFFFFFFFFFFFFDE
:1042A000FFFFFFFFFFFFFFFFFFFFFFCFFFFFFFF35A
:1042B000FFFFFFF3FFFFFFCFFFFFFF3FFFFFFF3FCA
:1042C000FFFFFFCFFFFFFFFFFFFFFFFFFFFFFFFF2E
:1042D000FFFFFFFFFFFFFFFFFFFFFFFFFFFFFFFFEE
:1042E000FFFFFFFFFFFFFFFFFFFFFFFCF003FFFFEC
:1042F000FFFFFFFFFFFFFFFCF003FCF003FCF003F8
:10430000FCF003FCF003FCF003FCF003FFFFFFF004
:10431000CCFFFF003FF0CCC3FF003FF0CCC3FFFF5A
:10432000FFFFFFFFFF0C3FFF33CFF033C3FFC3CFCF
:10433000FFFFFFFFFFFFFFFFFFFFF3CFFFF333FFA1
:1043400033CFFCCCFFFF3CFFFFFFFFFFFFFFFF0F62
:10435000FFFCF0FFFCCF3FFF3F3FFCCFFFFFFFFF25
:10436000FFFFFFFFFFFFFFFFFFFFFCF3FFFFFFFF6C
:10437000FFFFFFFFFFFFFFFFFFFFFFFFFFFFFCFF50
:104380003FC3FFC3FFFFFFFFFFFFFFFFFFFFFFFF75
:10439000C3FFC3FCFF3FFFFFFFFFFFFFFFFFFFFF68
:1043A000FFFFFFFFCFFFF0CFFFFF03FFF0CFFFFFC7
:1043B000CFFFFFFFFFF3FFFFF3FFFFF3FFFC000F53
:1043C000FFF3FFFFF3FFFFF3FFFFFFFFFFFFFFC35D
:1043D000FFFFF03FFFFF3FFFFFFFFFFFFFFFFFFF7C
:1043E000FFFFF3FFFFF3FFFFF3FFFFF3FFFFF3FF19
:1043F000FFFFFFFFFFFFFFFFFFFC3FFFFC3FFFFF53
:10440000FFFFFFFFFFFFFFFFFFFFFFF3FFFFFC3F8B
:10441000FFFFC3FFFFFC3FFFFFC3FFFFFFFFFFFFE7
:10442000FF000FFCFFF3FCFFF3FCFFF3FF000FFFA7
:10443000FFFFFFFFFFFCFFFFFCFFF3FC0003FCFF9F
:10444000FFFCFFFFFFFFFFFFFFFFFC3FCFFCCFF3B1
:10445000FCF3F3FCFCF3FC3F0FFFFFFFFFFFFFFF4C
:104460003FCFFCFFF3FCFCF3FCFCF3FF030FFFFF6B
:10447000FFFFFFFFFFC3FFFFCCFFFFCF0FFCCFF31A
:10448000FC0003FCCFFFFFFFFFFF3FFFFCFC03FC32
:10449000FCF3FCFCF3FF03F3FFFFFFFFFFFFFF0054
:1044A0003FFCFCCFFCFCF3FCFCF3FF03F3FFFFFF3E
:1044B000FFFFFFFFFFC3FFFFF3FC3FF3FFC0F3FF6E
:1044C000FF03FFFFFFFFFFFFFF030FFCFCF3FCFCFC
:1044D000F3FCFCF3FF030FFFFFFFFFFFFFFCFC0FEC
:1044E000FCF3F3FCF3F3FF33F3FFC00FFFFFFFFF19
:1044F000FFFFFFFFFFFC3C3FFC3C3FFFFFFFFFFFD8
:10450000FFFFFFFFFFFFFFFFFFFFF0FFFFFC3CCFC0
:10451000FF3CCFFFFFFFFFFFFFFFF3FFFFCCFFFFDD
:10452000CCFFFF3F3FFCFFCFFCFFCFFFFFFFFFFFB4
:10453000FFFFCCFFFFCCFFFFCCFFFFCCFFFFCCFF8A
:10454000FFFFFFFCFFCFFCFFCFFF3F3FFFCCFFFF94
:10455000CCFFFFF3FFFFFFFFFFFFFFFFFFFFFCFFAD
:104560003FFCFFCFFFF3CFFFFC3FFFFFFFFFFFFF4D
:10457000FC0003F3FFFCF3F0FCF3CF3CFCC003FFB3
:10458000FFFFFCFFFFFC0FFFFCC033FFCFC3FCC0ED
:104590003FFC0FFFFCFFFFFCFFF3FC0003FCFCF300
:1045A000FCFCF3FCFCF3FF030FFFFFFFFFFFFFFF2B
:1045B000000FFCFFF3FCFFF3FCFFF3FF3FC3FFFF23
:1045C000FFFCFFF3FC0003FCFFF3FCFFF3FF3FCF16
:1045D000FFC03FFFFFFFFCFFF3FC0003FCFCF3FC0C
:1045E000F033FCFFF3FC3FC3FFFFFFFFFFFFFCFFC7
:1045F000F3FC0003FCFCF3FFF033FFFFF3FFFFC30A
:10460000FFFFFFFF000FFCFFF3FCF3F3FF03C3FF0B
:10461000F3FFFFFFFFFCFFF3FC0003FCFCF3FFFCD8
:10462000FFFCFCF3FC0003FCFFF3FFFFFFFCFFF3C8
:10463000FCFFF3FC0003FCFFF3FCFFF3FFFFFFFFB5
:10464000FFFFFF03FFFCFFF3FCFFF3FF0003FFFF8F
:10465000F3FFFFFFFCFFF3FC0003FCF3F3FFF0FFAD
:10466000FFCF33FC3FC3FCFFF3FFFFFFFCFFF3FC76
:104670000003FCFFF3FCFFFFFC0FFFFFFFFFFCFF4D
:10468000F3FC0003FCFF03FFF0FFFCFF03FC00034F
:10469000FCFFF3FCFFF3FC0003FCFF03FFC0FFFC87
:1046A0003FF3FC0003FFFFF3FFFFFFFF000FFCFFE2
:1046B000F3FCFFF3FCFFF3FF000FFFFFFFFFFFFF23
:1046C000FCFFF3FC0003FCF3F3FFF3F3FFFC0FFF2D
:1046D000FFFFFFFFFFFF000FFCFFF3F0FFF3F0FF12
:1046E000F3F3000FFFFFFFFCFFF3FC0003FCF3F309
:1046F000FFF3F3FFC3F3FF3C0FFCFFFFFFFFFFFCE3
:104700003F0FFF3CF3FCFCF3FCFCCFFF03C3FFFFB8
:10471000FFFFFFC3FFFFF3FCFFF3FC0003FCFFF30D
:10472000FFFFF3FFFFC3FFFFF3FF0003FCFFF3FCFA
:10473000FFFFFCFFF3FF0003FFFFF3FFFFF3FFFFAB
:1047400003FFC0F3FC3FFFFFC0F3FFFF03FFFFF3D6
:10475000FFFFF3FF0003FCFFF3FF00FFFCFFF3FF8D
:104760000003FFFFF3FCFFF3FC3FC3FFCF3FFFF06D
:10477000FFFFCF3FFC3FC3FCFFF3FFFFF3FFFFC38F
:10478000FCFC33FC03FFFCFC33FFFFC3FFFFF3FF24
:10479000FFFFFC3FC3FCCFF3FCF0F3FCFF33FC3F17
:1047A000C3FFFFFFFFFFFFFFFFFFC00003CFFFF3CB
:1047B000CFFFF3FFFFFFFFFFFFFFFFFFFFFFF3FF51
:1047C000FC0FFFC3FFF03FFFFFFFFFFFFFFFFFFFF7
:1047D000FFFFFFFFCFFFF3CFFFF3C00003FFFFFF9B
:1047E000FFFFFFFFFFFFFFFCFFFFFF3FFFFFC3FFD8
:1047F000FF3FFFFCFFFFFFFF3FFFFF3FFFFF3FFFCC
:10480000FF3FFFFF3FFFFF3FFFFF3FFFFFFFFFFFB8
:10481000FFFFFFFFFFFFFFFFF3FFFFCFFFFFFFFFE4
:10482000FFFFFFFFFFFF0CFFFCF33FFCF33FFCF338
:104830003FFC00FFFCFFFFFCFFF3FC0003FCFCFF60
:10484000FCFF3FFCFF3FFF00FFFFFFFFFFFFFFFFFD
:1048500000FFFCFF3FFCFF3FFCFF3FFF3C3FFFFF33
:10486000FFFFFFFFFF00FFFCFF3FFCFF3FFCFCF3EF
:10487000FC0003FCFFFFFFFFFFFF00FFFCF33FFC1A
:10488000F33FFCF33FFCF0FFFFFFFFFFFFFFFCFFE8
:104890003FFC000FFCFF33FCFF33FCFF33FFFFFF47
:1048A000FFFFFFFF00FFCCFF3FCCFF3FCCFCFFF042
:1048B000003FFFFF3FFCFFF3FC0003FCFCFFFFFF9A
:1048C0003FFCFF3FFC00FFFCFFFFFFFFFFFCFF3F43
:1048D000FCFF3FFC0033FCFFFFFCFFFFFFFFFFFF7F
:1048E000FFFFCFFF3FCFFF3FCFFF33F0003FFFFF82
:1048F000FFFFFFFFFCFFF3FC0003FFF3FFFCC33FE0
:10490000FC3C3FFCFF3FFFFFFFFFFFFFFCFFFFFC06
:10491000FFF3FC0003FCFFFFFCFFFFFFFFFFFCFFBA
:104920003FFC003FFCFF3FFC00FFFCFF3FFC00FFA3
:10493000FCFFFFFCFF3FFC003FFCFCFFFFFF3FFCD8
:10494000FF3FFC00FFFCFFFFFFFFFFFF00FFFCFF3E
:104950003FFCFF3FFCFF3FFF00FFFFFFFFCFFF3F9C
:10496000C0003FCCFCFFFCFF3FFCFF3FFF00FFFF10
:10497000FFFFFFFFFFFF00FFFCFF3FFCFF3FCCFC02
:10498000FFC0003FCFFF3FFFFFFFFCFF3FFC003FAA
:10499000FCFCFFFCFF3FFCFF3FFFFFFFFFFFFFFCB6
:1049A0003CFFFCF33FFCF33FFCF33FFF0C3FFFFFFA
:1049B000FFFFFFFFFFFF3FFF000FFCFF3FFCFF3F3C
:1049C000FCFF3FFF3FFFFFFF3FFF003FFCFFFFFCFF
:1049D000FFFFFF3F3FFC003FFCFFFFFFFF3FFFF0FB
:1049E0003FFF0F3FFCFFFFFF0F3FFFF03FFFFF3F89
:1049F000FFFF3FFF003FFCFF3FFF03FFFCFF3FFFC8
:104A0000003FFFFF3FFCFF3FFC3C3FFFC3FFFFC3F6
:104A1000FFFC3C3FFCFF3FFFFFFFFFFF3FCFFC3FA2
:104A2000CFC33FC03FFFCF0F3FFFF03FFFFF3FFF30
:104A3000FFFFFC3C3FFCCF3FFCF33FFCFC3FFC3F57
:104A40003FFFFFFFFFFFFFFFFFFFFFCFFFF0300F34
:104A5000CFFFF3FFFFFFFFFFFFFFFFFFFFFFFFFFA2
:104A6000FFFFF00003FFFFFFFFFFFFFFFFFFFFFF60
:104A7000FFFFFFFFCFFFF3F0300FFFCFFFFFFFFF80
:104A8000FFFFFFFFFFFFFFCFFFFFF3FFFFCFFFFFA2
:104A9000CFFFFFF3FFFFFFFFFFFFFFFFFFFFFFFF62
:104AA000FFFFFFFFFFFFF300FFFFFFFFFFFFFFF030
:104AB000FFFFFFF0FFFFCCCFF003CCCCF003FCCC2A
:104AC000FFFFF3CFC300FC33FFFFFFFFFF3FFF30CB
:104AD000F0CFFFCFFFFFF03FF303F0F3F3F3FFFF5F
:104AE000FFFFFFC0FFFFFFFFFFFFFFFFF003CFFC53
:104AF000FFFFFFFFCFFCF003FFFFFFFFFFFFFF33D0
:104B0000FFC0FF33FFFFFF3FFF3FF003FF3FFF3FCB
:104B1000FFFFFFFFC3FFFCFFFFFFFFFFFF3FFF3F64
:104B2000FF3FFFFFFFFFFFFFF3FFFFFFFFFFCFFF91
:104B3000F0FFFF03FFFCFFFFFFFFFC03F3FCFC03A0
:104B4000FFFFF3FFF3FCF000F3FFF3FFFFFFF0F3D1
:104B5000F33CF3C3FFFFFFFFF3F3F33CFCC3FFFFA2
:104B6000FFFFFF0FF333F000F33FFFFFFCC0F3CC78
:104B7000FC3CFFFFFFFFFC03F3CCFC3CFFFFFFFF0F
:104B8000FFF0F03CFFC0FFFFFFFFFC33F3CCFC3332
:104B9000FFFFFFFFF3C3F33CFC03FFFFFFFFFFFF3B
:104BA000F3CFFFFFFFFFFFFFFFFFF3FFFCCFFFFF90
:104BB000FF3FFF3FFCCFF3F3FFFFFFFFFF33FF3368
:104BC000FF33FFFFFFFFF3F3FCCFFF3FFF3FFFFF8C
:104BD000FFF3F33CFFC3FFFFFFFFF003CFFCCF3C2D
:104BE000CC03F0FFF30CFF30F30FF0FFF3FCF00009
:104BF000F3CCF3CCFC33FFFFFC00F3FCF3F0FFFF3E
:104C0000F3FCF000F3FCF3FCFC03F3FCF000F3CC4A
:104C1000F3FCF0F0F3FCF000F3CCFFFCFFF0FFFF3F
:104C2000FC03F3FCF03CFF3FF3FCF000F3CCFFCFC0
:104C3000F000FFFFF3FCF000F3FCFFFFFFFFFC3F81
:104C4000F3FCFC00FFFCF3FCF000FF0FF030F3FC82
:104C5000F3FCF000F3FCF3FFF0FFF000F3C0FF3FC4
:104C6000F3C0F000F3FCF000F3C3FC3CF000FFFFE6
:104C7000FC03F3FCF3FCFC03F3FCF000F33CFF3C0F
:104C8000FFC3FFFFFC03F3FCF0FCF000F3FCF000BB
:104C9000F33CFF3CF0C3FFFFF3F0F3CCF030FFFF39
:104CA000FFF0F3FCF000F3FCFFF0FFFCFC00F3FF6F
:104CB000F3FCFC00FFF0FC0CF3FFF03CFFC0FC0039
:104CC000F3FCFC0FF3FCFC00F3FCF0F0FF0FF0F042
:104CD000F3FCFFF0F3CCF03FF3CCFFF0FFFFF0F07C
:104CE000F33CF3CCF0F0FFFFFFFFC000CFFCFFFF71
:104CF000FFFCFFC3F03FCFFFFFFFFFFFCFFCC00073
:104D0000FFFFFFFFFFFFFFCFFFF0FFCFFFFF3FFFE2
:104D10003FFF3FFF3FFFFFFFFFFFFFFFFFFCFFF3F2
:104D2000FFFFFFFFF0FFF0CFF00FF3FFF3FCF00009
:104D3000F3CFF3CFFC3FFFFFF00FF3CFF3CFFFFF35
:104D4000FFFFFC3FF3CFF3CCF000FFFFFC0FF30FAE
:104D5000F30FFFFFFFFFF3CFF003F3CCFFFFFFFFE5
:104D6000FC3F33CF33CFC00FF3FCF000F3CFFFCFC6
:104D7000F03FFFFFF3CFF00CF3FFFFFFFFFF3FCF4C
:104D80003FCC000FFFFFF3FCF000FF3FF00FF3CF2D
:104D9000FFFFF3FCF000F3FFFFFFF00FFFCFF03F4A
:104DA000FFCFF03FF3CFF00FFFCFFFCFF03FFFFF7C
:104DB000FC3FF3CFF3CFFC3F3FCF000F33CFF3CF18
:104DC000FC3FFFFFFC3FF3CF333F000FFFFFF3CF6C
:104DD000F00FF3CFFFCFFFFFF3FFF30FFCCFFFFF89
:104DE000FFCFFC03F3CFF3CFFCFFFFCFFC0FF3FFAC
:104DF000F3CFF00FFFCFFF0FF0FFF0FFFF0FFC0F1F
:104E0000F3CFFC3FF3CFFC0FFFFFF3CFFC3FFC3FA2
:104E1000F3CFFFCF3C0F03FFFC0FFFCFFFFFF3CF1C
:104E2000F0CFF30FF3CFFFFFFF3FF003CFFCFFFF07
:104E3000FFFFFFFFC000FFFFFFFFFFFFCFFCF003FE
:104E4000FF3FFFFFFFFFFCFFFF3FFCFFFF3F820034
:104E50000000AA000000AAAA0000AAAAAA0055AA57
:104E6000AA0055555555AAAAAAAA55555555AAAAF4
:104E7000AAAA151515150505050501010101000072
:104E80000000000000000000000000000000000022
:104E9000000000000000000000000000000041458C
:104EA000F1FF5F5501000000C84E0008000000201F
:104EB000DC0100004A030008684F0008DC01002004
:104EC000CC06000004010008120C0A28F003121C92
:104ED00013F03813F07013F0E01008F0C001F08008
:104EE00003F01307F0130EF0131CF01338F01370D7
:104EF000F013E0F013C0F12380F322F722F60A1337
:104F0000F003092B7509A00381400A030406080C6D
:104F1000101820302D0102030404350607080994F7
:104F200080841E6917B930120432503904137F1877
:104F300013080E12051379321B080B1913CD4213F7
:104F40000807120313984A13080592021345161C0A
:104F5000084F171C19041AF10C1321141B084108DF
:084F60001A3D041A370C000091
:0400000508000149A5
:00000001FF
